:020000040000FA
:040000006B303A28FF
:08000800A000030EA100831209
:1000100005191028831601178312B23081002B288E
:1000200083160113831203140B190310A80DA90DD5
:10003000AA0DAB0DAC0DAC16FF302C02031D2B2806
:10004000FA302B02031D2B2831152A08AF0029088E
:10005000AE002808AD008B100B11210E8300A00EFE
:04006000200E090065
:0C007400203084008001840A6030040207
:10008000031C3C281230B00083218316FF2390000C
:10009000831283160C308505870183128501870141
:1000A000073099000030831691009F008312C830FA
:1000B00083168100831231309000003083168C004B
:1000C000831210308B00CE2181018E018F010B1124
:1000D0008B100B108C018B177B2031197E20B30BFA
:1000E0007928031085190314B90DF030390203196A
:1000F0000A21E7216C286400321008003111013018
:10010000B7008B132030370783169B001C141A0886
:100110008312A4001030370783169B001C141A08A2
:100120008312A300A6000230A6060030370783160C
:100130009B001C141A088312A200A7000130A70616
:100140008B17321CA92822090339A200A309A4098C
:10015000A50924082F02031D042923082E02031DCC
:10016000D82822082D02031D042901303702031D5F
:10017000BC283D143E14972102303702031DC328CA
:10018000BD143E149B2103303702031DCA283D15C0
:100190003E149F2104303702031DD128BD153E14A3
:1001A000A32105303702031DD8283D163E14A72190
:1001B00026082E02031D042927082D02031D0429E9
:1001C00001303702031DE7283D103E14AB210230F9
:1001D0003702031DEE28BD103E14AF210330370255
:1001E000031DF5283D113E14B32104303702031DD1
:1001F000FC28BD113E14B72105303702031D032929
:100200003D123E14BB210429B70A063037020318F9
:10021000080081280130B600B300B400B500B70073
:1002200085018701B1137B20B30B36290310851993
:100230000314B90DF030390203195D29B40B3629C6
:10024000013037020319BF21023037020319C221DE
:10025000033037020319C521043037020319C821BE
:10026000053037020319CB219630B400311D132914
:100270003111321C40292D090339AD00AE09AF09F7
:100280002F1C13298E018F010C1C13290C102E1EFC
:1002900013298B1320303707BB002F08BA007021B9
:1002A00010303707BB002E08BA0070210030370726
:1002B000BB002D08BA0070218B1785018701B70A92
:1002C000B60106303702031C1329CE2108003E1C5C
:1002D00008003E101030BB003D08BA007021080035
:1002E0008B133A0883161C159A003B089B00553067
:1002F0009D00AA309D009C1464009C187C291C1150
:1003000083128B170800831610309B001C141A08E8
:100310008312BD00FF30D000D415D515D615D715E2
:10032000D815D915DA15DB15DC15DD150800D21046
:100330004E14CE100800D2114E15CE110800D21264
:100340004E16CE120800D2134E17CE130800D3104B
:100350004F14CF1008005210CE144E100800521146
:10036000CE154E1108005212CE164E12080052132E
:10037000CE174E1308005310CF144F100800303022
:100380008506080003308506080006308706080049
:100390002130870608001830870608003D184E14E3
:1003A0003D1CCE14BD184E15BD1CCE153D194E1664
:1003B0003D1DCE16BD194E17BD1DCE173D1A4F144B
:1003C0003D1ECF144E08D2004F08D30008008F08FE
:1003D000031908008F01D00F292BD00A521CFF29C6
:1003E000541DF529D40154160D2AD41DFA29D4011F
:1003F00054160D2A541E0D2AD401D4140D2AD41CCF
:10040000042AD40154150D2A541D092AD401D415E7
:100410000D2A541E0D2AD4015415D21C1E2A551D16
:10042000142AD50155162C2AD51D192AD501551681
:100430002C2A551E2C2AD501D5142C2AD51C232A4A
:10044000D50155152C2A551D282AD501D5152C2A3C
:10045000551E2C2AD5015515521D3D2A561D332AED
:10046000D60156164B2AD61D382AD60156164B2AC7
:10047000561E4B2AD601D6144B2AD61C422AD60128
:1004800056154B2A561D472AD601D6154B2A561EFD
:100490004B2AD6015615D21D5C2A571D522AD70168
:1004A00057166A2AD71D572AD70157166A2A571E88
:1004B0006A2AD701D7146A2AD71C612AD70157158F
:1004C0006A2A571D662AD701D7156A2A571E6A2A33
:1004D000D7015715521E7B2A581D712AD80158166C
:1004E000892AD81D762AD8015816892A581E892AA1
:1004F000D801D814892AD81C802AD8015815892AED
:10050000581D852AD801D815892A581E892AD8014C
:100510005815D21E9A2A591D902AD9015916A82A6F
:10052000D91D952AD9015916A82A591EA82AD901D8
:10053000D914A82AD91C9F2AD9015915A82A591DAE
:10054000A42AD901D915A82A591EA82AD9015915B2
:10055000521FB92A5A1DAF2ADA015A16C72ADA1DC4
:10056000B42ADA015A16C72A5A1EC72ADA01DA143F
:10057000C72ADA1CBE2ADA015A15C72A5A1DC32A0D
:10058000DA01DA15C72A5A1EC72ADA015A15D21F0C
:10059000D82A5B1DCE2ADB015B16E62ADB1DD32A97
:1005A000DB015B16E62A5B1EE62ADB01DB14E62A8A
:1005B000DB1CDD2ADB015B15E62A5B1DE22ADB0181
:1005C000DB15E62A5B1EE62ADB015B15531CF72AC6
:1005D0005C1DED2ADC015C16052BDC1DF22ADC011A
:1005E0005C16052B5C1E052BDC01DC14052BDC1CCA
:1005F000FC2ADC015C15052B5C1D012BDC01DC15E4
:10060000052B5C1E052BDC015C15D31C162B5D1D18
:100610000C2BDD015D16242BDD1D112BDD015D167C
:10062000242B5D1E242BDD01DD14242BDD1C1B2B54
:10063000DD015D15242B5D1D202BDD01DD15242B37
:100640005D1E242BDD015D1567214E08D2004F0889
:10065000D3005008D1000C305405031D05120C3096
:100660005505031D85120C305605031D05100C3071
:100670005705031D85100C305805031D87100C30DD
:100680005905031D07110C305A05031D07100C30C6
:100690005B05031D87120C305C05031D07120C302F
:1006A0005D05031D871151080E020318832B1230BC
:1006B0005405031D051612305505031D851612300D
:1006C0005605031D051412305705031D85141230FD
:1006D0005805031D871412305905031D07151230E4
:1006E0005A05031D071412305B05031D87161230CF
:1006F0005C05031D071612305D05031D8715FF30CD
:100700005002031908008F08031D08007B205108C0
:100710000E02031C832B18305405031D05120630EE
:100720005405031D051618305505031D85120630A6
:100730005505031D851618305605031D0510063096
:100740005605031D051418305705031D8510063086
:100750005705031D851418305805031D87100630F2
:100760005805031D871418305905031D071106305D
:100770005905031D071518305A05031D07100630CB
:100780005A05031D071418305B05031D8712063038
:100790005B05031D871618305C05031D0712063024
:1007A0005C05031D071618305D05031D8711063013
:0807B0005D05031D871508001B
:084000000200030006000200AB
:02400E00CC01E3
:10420000010078007A007C007E007B0079007F004E
:104210007D007A0078007E007C00FF00FF00FF0038
:104220000000F200F600FA00FE00F200F600FA00CC
:10423000FE00F200F600FA00FE00FF00FF00FF00A3
:10424000010005000500050005000900090009003E
:1042500009000D000D000D000D00FF00FF00FF0024
:10426000FF00FF00FF00FF00FF00FF00FF00FF0056
:10427000FF00FF00FF00FF00FF00FF00FF00FF0046
:10428000FF00FF00FF00FF00FF00FF00FF00FF0036
:10429000FF00FF00FF00FF00FF00FF00FF00FF0026
:1042A000FF00FF00FF00FF00FF00FF00FF00FF0016
:1042B000FF00FF00FF00FF00FF00FF00FF00FF0006
:1042C000FF00FF00FF00FF00FF00FF00FF00FF00F6
:1042D000FF00FF00FF00FF00FF00FF00FF00FF00E6
:1042E000FF00FF00FF00FF00FF00FF00FF00FF00D6
:1042F000FF00FF00FF00FF00FF00FF00FF00DD00E8
:00000001FF
